:1000000011C020C01FC01EC01DC01CC01BC01AC014
:1000100019C018C017C016C015C014C013C06E6F29
:100020006465200011241FBECFE5D1E0DEBFCDBF47
:1000300020E0A0E6B0E001C01D92A436B207E1F7CF
:100040003BD16FC1DDCFFC01DA011C929081962378
:10005000E9F785E88A95F1F7000087EC90E00197D1
:10006000F1F700C000008081862319F08C91816037
:100070008C9387EC90E00197F1F700C0000080813D
:10008000862319F08C9182608C9387EC90E0019725
:10009000F1F700C000008081862319F08C91846004
:1000A0008C9387EC90E00197F1F700C0000080810D
:1000B000862319F08C9188608C9387EC90E00197EF
:1000C000F1F700C000008081862319F08C918061D7
:1000D0008C9387EC90E00197F1F700C000008081DD
:1000E000862319F08C9180628C9387EC90E00197C5
:1000F000F1F700C000008081862319F08C918064A4
:100100008C9387EC90E00197F1F700C000008081AC
:10011000682319F08C9180688C9387EC90E00197AC
:10012000F1F700C0000095E89A95F1F700000895F6
:10013000FC019081862F809598239083A7ECB0E0F6
:100140001197F1F700C0000040FF04C09081962B8A
:10015000908303C0908198239083A7ECB0E011971F
:10016000F1F700C0000041FF04C09081962B9083FE
:1001700003C0908198239083A7ECB0E01197F1F72A
:1001800000C0000042FF04C09081962B908303C002
:10019000908198239083A7ECB0E01197F1F700C00D
:1001A000000043FF04C09081962B908303C0908190
:1001B00098239083A7ECB0E01197F1F700C00000FE
:1001C00044FF04C09081962B908303C090819823B4
:1001D0009083A7ECB0E01197F1F700C0000045FF55
:1001E00004C09081962B908303C0908198239083C4
:1001F000A7ECB0E01197F1F700C0000046FF04C083
:100200009081962B908303C0908198239083A7ECD4
:10021000B0E01197F1F700C00000442324F480817E
:10022000862B808303C090818923808387EC90E0B4
:100230000197F1F700C000008081682B6083A7EC74
:10024000B0E01197F1F700C0000087EC90E0019753
:10025000F1F700C000000895CF93DF93EA011092F8
:10026000630010926200E0916200F0916300EC0F75
:10027000FD1F44914093610060E188E390E058DF06
:100280008091620090916300019690936300809347
:100290006200809161008111E6CFDF91CF910895D6
:1002A000C0982FEF80E792E0215080409040E1F726
:1002B00000C00000C09A089580E886BD16BCC49AAC
:1002C000BC98C09AB89A40E650E068E086E390E0B7
:1002D000BADEE6DF809160008033A9F7BC9A4EE178
:1002E00050E060E188E390E0B7DF4091600060E1BA
:1002F00088E390E01DDF4AE060E188E390E018DFEA
:100300002FEF80E792E0215080409040E1F700C05D
:100310000000C6DFC5DFC4DFC3DFC2DFC1DFBC98BA
:06032000D2CFF894FFCFDC
:00000001FF
